:100000000C94340018950000189500001895000015
:10001000189500001895000018950000189500002C
:10002000189500001895000018950000189500001C
:10003000189500001895000018950000189500000C
:1000400018950000189500000C943F0318950000C7
:1000500018950000189500001895000018950000EC
:1000600018950000189500008FEF8DBFC0EEE8E7EF
:100070004E2E84E08EBFD4E0F4E05F2EEEEFF3E08E
:10008000A0E0B1E088278D933197E9F78FEC80935A
:10009000C40080E08093C50088E18093C10066249D
:1000A0007091C10070687093C1003898229A87E0FF
:1000B00085B98FE188B9789482E38093870282E3DF
:1000C00090E00E94F6022A9882E390E00E94F602F5
:1000D0002A9AA7E8B2E08C9181508C930091870214
:1000E000003011F00C945F002A980027A6E2B0E0DF
:1000F0008C9180FB0EF401E041E0041711F00C94A8
:1001000083000C94860087E68093C4000E94DD0281
:10011000ECEBF7E00E94D6020E94DD020E94DD02B5
:10012000E1E0F0E00E94E7022A9A88EC90E00E9469
:10013000F6022A988FEC8093C40080E0809334020A
:1001400081E0809330020E94A502A8E0B1E08C9388
:1001500000910801043211F00C94B7000E94BA0318
:10016000A9E0B1E034E60E948C020E94B70381E06E
:10017000E9E0F1E005E00A93A3EDB1E00E948E030F
:10018000A3EDB1E0ECEEF7E00E94A30311F00C94B4
:10019000A3002A9AE9E0F1E0A1EEB1E09CE20CE0D4
:1001A00036E00E94BF03AFE2B2E02C9381E080937F
:1001B000300240912F0200913002041718F011F024
:1001C0000C94EA00A0E3B2E08C918F5F8C9310F462
:1001D0000C94D900EEEEF1E0ACE4B2E00E948903A9
:1001E000EBEFF1E0A9E5B2E00E948903E8E0F2E07C
:1001F000ACE5B2E00E948903E5E1F2E0A9E6B2E0F5
:100200000E948903E2E2F2E0ACE6B2E00E948903D8
:10021000ACE6B2E0E2EFF7E02FEF91E00E941003CE
:10022000A2E8B2E00C93A2E8B2E08C9181508C93EA
:10023000ECE6F2E000918202ACE6B2E00E949503A7
:10024000ACE6B2E00E949D03A3E8B2E08C9300917B
:100250008302043011F00C943501ACE6B2E00E9448
:100260008302E4EFF7E00E9405030091830205306A
:1002700011F00C944301ACE6B2E00E948302EAEF75
:10028000F7E00E94050300918302063011F00C9400
:100290005101ACE6B2E00E948302E0E0F8E00E9487
:1002A000050300918302073011F00C945F01ACE666
:1002B000B2E00E948302E4E0F8E00E9405030091AE
:1002C0008302083011F00C946D01ACE6B2E00E949C
:1002D0008302E8E0F8E00E940503ACE6B2E0EAE061
:1002E000F8E02FEF91E00E941003A4E8B2E00C9335
:1002F0000091840241E0041BA5E8B2E00C9309E000
:1003000040918402041BA6E8B2E00C9300918302A2
:10031000093011F00C94AE01ECE6F2E00091850298
:10032000A7E7B2E00E949503ACE6B2E00E949D030D
:10033000EA2FFB2F009186023197E01BF0400FEF70
:10034000A7E7B2E00E9483020E949503A7E7B2E00C
:100350000E948302E8E0F8E00E9405030091830216
:10036000093011F00C94BA01E7E7F2E0ACE6B2E034
:100370000E948903AEE6B1E0ECE0F8E00E940503DC
:10038000ECE4F2E0AEE6B1E00E9483020E94890351
:10039000AEE6B1E00E948302E8E0F8E00E940503C7
:1003A000E9E5F2E0AEE6B1E00E9483020E94890333
:1003B000AEE6B1E00E948302E8E0F8E00E940503A7
:1003C000ECE5F2E0AEE6B1E00E9483020E94890310
:1003D000AEE6B1E00E948302E8E0F8E00E94050387
:1003E000E9E6F2E0AEE6B1E00E9483020E948903F2
:1003F000AEE6B1E00E948302E0E2F8E00E9405036D
:10040000AEE6B1E00E949D03A5E3B2E08C9381E0EB
:10041000809330024091350200913002041718F0A9
:1004200011F00C94310280913002EEE6F1E001E02F
:100430000A93A6E3B2E00E948E03009134020F9368
:10044000A6E3B2E08C91482F0F910427A4E3B2E019
:100450000C93A0E3B2E08C918F5F8C9310F40C941A
:100460000A020027A6E2B0E08C9180FB0EF401E0C6
:1004700041E0041711F00C943F020C94420287E60D
:100480008093C400A0E6B4E0E6E3F8E00E94050330
:10049000EEE6F1E0A0E6B4E00E9483020E94890348
:1004A000A0E6B4E00E948302E2EFF7E00E940503B9
:1004B000A0E6B4E00E948302E4E3F2E00E946D0350
:1004C0000E94CE020E94DD02ACE6B2E00E94D002A1
:1004D0000E94DD0284E690E00E94F6022A98A9E0DC
:1004E000B1E088278C93AEE6B1E088278C93ACE628
:1004F000B2E088278C93A7E7B2E088278C930C940E
:100500009A00F894FFCF8F938D918823E9F7119784
:100510008F910895A0E6B4E01DD0883091F08D3021
:1005200039F03323C9F38D933A9563FE49D0F4CF64
:1005300063FC04C08DE044D08AE042D088278C93CD
:1005400008953ED011973395E7CF8091EE0288232E
:1005500009F408950F929F93AF93BF937F93809177
:10056000EE028823E1F3F8948091EE028A9580935D
:10057000EE029091EC02A8E8B2E0A90F0024B01DB1
:100580008C919395943609F499279093EC02789482
:100590007F91BF91AF919F910F900895A0E6B4E035
:1005A0008D91882311F00CD0FBCF08950E943B035E
:1005B000802D11F005D0FACF08958DE001D08AE0AA
:1005C0000090C00005FEFCCF8093C600089588EE21
:1005D00093E00CD03197D9F708953197F1F708954A
:1005E000689462F80895E89462F80895EF93FF9391
:1005F000EE27E82BE92B31F0E0EAFFE03197F1F745
:100600000197D1F7FF91EF9108950E943B030D925E
:100610000020D9F7089599910027A90FB01F1197CD
:10062000492F4A955E2F6F2FE8941127439520306C
:1006300019F0C895802D01C080818823B9F07C9184
:100640007723A1F0781739F40EF0042F13956894EE
:1006500011963196EBCF112321F0411BA11B1127DD
:10066000B10BE894E52FF62F1196E0CF882311F017
:10067000002708950895C8953196002008957F9326
:100680000F93AF93BF938F939F938FB78F93809167
:10069000EE0204E6081B29F49091C6000E94F002C5
:1006A00013C00091ED02A8E8B2E077279091C60050
:1006B000A00FB71F9C9383958093EE020395043699
:1006C00009F400270093ED028F918FBF9F918F91C6
:1006D000BF91AF910F917F91189541E003C042E027
:1006E00001C044E0E40F8827F81F8291982F82957B
:1006F00006D0892F04D04A95C1F70C9486038F70D9
:100700008A3008F0895F805D8D93089588278D93E6
:10071000089581918D938823E1F70895099191912E
:10072000992351F08A95D9F7319781918D930A9544
:1007300019F08823D1F70895E9CF8FEF83959D9124
:100740009923E1F70895689401C0E894AF93BF93AB
:100750008D9116F0919103C00E943B03902D891753
:1007600018F011F48823A1F7BF91AF910895E89490
:1007700063F80895689463F80895689401C0E89454
:100780002227102F231709F4089526F40E943B0313
:10079000802D01C08191803051F0891731F08D9307
:1007A0001A9599F723951D93ECCF01D0EACF2395A5
:1007B000882713958D931A95E9F7089557504C3271
:1007C00044524154532056657273696F6E20332E24
:1007D000312020202020284329444A374F4F4054BD
:1007E0002D4F4E4C494E452E444500004750575022
:1007F0004C002A00202020202C002020202C00004B
:1008000020202C00202C00002C002D004750524DA1
:10081000432C3132333435362E3030302C412C00DD
:100820002C312E30302C3130302E30302C303130D5
:080830003130302C2C002400B3
:00000001FF
